:030000000219FDE5
:03000B000200A848
:03002B0002015A75
:03005B000202EEB0
:030073000202DBAB
:1000800002030406080C10182030406080040608A3
:100090000C10182030406080A0C00003070F1F051F
:1000A000050D050305030302C2AFC0D0C0E0206206
:1000B00014E5256009E473E525F4F58AD262D0E001
:1000C000D0D0D2AF3285268AC262E526F4602F30C6
:1000D000682520720DD0E0D0D0D295D293D297D29D
:1000E000AF32D295D293D297206F0C206609740656
:1000F000D5E0FDE57B4290D0E0D0D0D2AF32758A1A
:1001000000C28DD26201F701B7306805206602C2D5
:100110009501B7306805206602C29701B7306805BF
:10012000206602C29301B7C29430680A2066077441
:1001300006D5E0FDC29501B7C29630680A20660771
:100140007406D5E0FDC29701B7C29230680A2066F6
:10015000077406D5E0FDC29301B7C2AFC2AD53E646
:10016000EFC0D0C0E0D2D3D2AFC2CEE52A60072024
:100170007449152A21BB7800790020742EE580305F
:100180007E01F430E50278FF53DACF207E0343DAB4
:1001900020307E0343DA10C2D8C271E580307E0180
:1001A000F430E50279FFC3E89970CB306103752A1A
:1001B00018207403752A18885CD27020740DE52B02
:1001C0006004152B21CB43DA01C2D8207002413ED6
:1001D000A85C206102C270207431C3E894F040032F
:1001E00074F0F8E8C4540F28F87984B70302410B7F
:1001F000C313C3138721200802C313200A06C3C8F0
:1002000098F8410B28F8500374FFF8C3E89565503F
:1002100003E565F88822E52D54066022206B1FE572
:1002200036C333C333F8E564C313C313F9C395224C
:1002300040028922E82522F52250037522FF8522FB
:1002400024A824C3E52495614002A8618825E566B9
:1002500070024182C3E8AA669A5003E8FAE4F9EA18
:10026000C333FBE568F45B29400D2567F8E567605B
:10027000021567400B41820AC3E5679A5002056781
:1002800078FF8826C26FC3E52694F84002D26FC378
:10029000E52594404002D26420CF0AD0E0D0D0437C
:1002A000E610D2AD32C2CF053A7801E52A600530BA
:1002B0007402152AC3E55C94014005755F0041D1C5
:1002C000756000756900E55F2401F55F5003755F97
:1002D000FFD0E0D0D043E610D2AD32C2AF53E67FBC
:1002E0007592FA7593FFC260759104D2AF32C2AFB6
:1002F00053E6EFC2ADC0D0C0E0C0F0D2D3D2AFA8B9
:10030000FBA9FCC2D8307102615553DACF207E03BD
:1003100043DA10307E0343DA20D271E580307E016B
:10032000F420E502612C88278928A18253DACF20A6
:100330007E0343DA20307E0343DA10C2D8C2713024
:100340007402A16E7800E580307E01F430E502A1F0
:100350006E885CA15653DACF207E0343DA20307ECC
:100360000343DA10C271206102812E53DACF207E5E
:100370000343DA10307E0343DA20C2D8D2718857A3
:100380008958C3E89555F8E99556F97B007E087AB7
:1003900000C3E8948CE994005005755B00812088C7
:1003A0002178A2E6A8216055C3E894C8E9940050DA
:1003B00008E4D2E4FB7A0A61FBC3E89468E994019B
:1003C0005008E4D2E3FB7A0F61FBC3E894D0E994D0
:1003D000025008E4D2E2FB7A1E61FBC3E894A0E974
:1003E00094055008E4D2E1FB7A3C61FBC3E89498A1
:1003F000E994085008E4D2E0FB7A787E00C3E895DF
:1004000059FCE9955AFD30E70AECF42401FCEDF4BF
:100410003400FD755B00C3EC9AED9E5003755B01E3
:100420008859895A8557558558567802A156C3E888
:100430009527F8E99528F9307C02A13A307B02A192
:100440003A307A02A1332075028151E9FDE8FC813E
:1004500070E9C313F9E813F8307902A133E9C31343
:10046000F9E813F8307802A133E9C313FDE813FC6F
:0F04700020612CC3EC941CED940240028187EDB7
:10047F00701EC3EC94C850180529E5297002152980
:10048F00C3E529940A5002A16E755C00D270A16E6B
:10049F00E529600215297888E6F97400207F08782D
:1004AF0096B90302789EE624FAFEE43400FFC3EC0B
:1004BF009EFCED9FFD9208B90310A208500720760D
:1004CF0009D27681D9307602C276A2085016B903C6
:1004DF000DECF42401FCEDF43400FD0204F378007C
:1004EF007900A13AB90315EC33FCED33FDC3EC945D
:1004FF000AFCED9400FD50047C007D00C3EC94FFDA
:10050F00ED9400400678FF7900A13AEC8572F0A4D3
:10051F00C5F0A2F733F87900400302055678FF794A
:10052F0000020556E9C313F9E813F8307C0EE960B1
:10053F000278FFC3E81338F8E43400F9C3E894FFF6
:10054F00E99400400278FF885CD270206102A16EAE
:10055F00741FF4552F4BF52FC274EB7002D27475C4
:10056F002A18307403752A0A306102A1822074039D
:10057F0053DAFE207403752B06D0F0D0E0D0D0D222
:10058F00AD43E6103279010205B279030205B27963
:10059F000A0205B2791E0205B279640205B279C862
:1005AF000205B27817E4D5E0FDD8FAD9F6227A140D
:1005BF007B780205D97A107B8C0205D97A0D7BB432
:1005CF000205D97A0B7BC80205D97902E4C296D508
:1005DF00E0FDC297D5E0FDD297D5E0FDD296D5E0EC
:1005EF00FDE920E002C29530E002C293E573D5E049
:1005FF00FDE920E002D29530E002D2937496D5E067
:10060F00FDD9C9EAF8D5E0FDD8FBDBBEC29622C3FF
:10061F007C007D0075F00005F0EA33FAEB33FB50F8
:10062F00F6EB13FBEA13FAC3E9FFE8FEE89AF8E9E1
:10063F009BF95004EFF9EEF8B3EC33FCED33FDD535
:10064F00F0DFEDF9ECF822E889F08A20D2D4F8A98E
:10065F00F07B0030F70B7BFFF42401F8E9F4340052
:10066F00F9E88520F0A4ADF0F8E98520F0A4AFF00B
:10067F00FEED2EF974003FFA7C04C3EA13FAE91376
:10068F00F9E813F8DCF48BF030F70AE8F42401F8FA
:10069F00E9F43400F9E889F0C2D4F8A9F02222C3B2
:1006AF00E54113F9E54013F8C3E54498F8E545999A
:1006BF00F9500CC3E89480E994FF40160206E5C395
:1006CF00E8947FE9940050030206E5787F790002F1
:1006DF0006E5788079FF8849894A22E5492546F859
:1006EF00E54A3547F9854A20E4300701F43548FAE1
:1006FF0030E709C3EA94F04015020723C3EA940FC9
:10070F00500302072378FF79FF7A0F02072378003F
:10071F0079007AF0C3E5249561500AC374019524DA
:10072F00500B020741E54A20E70E020741E54A3028
:10073F00E706884689478A482278A5E6FAC3E5493D
:10074F0033F8E54A33F9D156E930E70BC3E8948023
:10075F00E994FF4013E17BC3E8947FE994005002D2
:10076F00E17B787F7900E17B788079FFE820E715DE
:10077F00C3E52398F84009C3E8940140030207A298
:10078F0078010207A2E8F424012523F840030207A9
:10079F00A278FF884B2278A6E6FAA847A948D15637
:1007AF00E930E70CC3E89401E994FF40160207D63D
:1007BF00C3E894FFE9940050030207D678FF79004D
:1007CF000207D6780179FFE920E715C3E54B98F8C2
:1007DF004009C3E8940140030207FD78010207FDB9
:1007EF00E8F42401254BF840030207FD78FF882425
:1007FF002278FFC26420693D206A12D264C3E541AA
:10080F00940A4009C3E52594405002C26479A1E7D8
:10081F006023E541601F74FF8541F0848539F03016
:10082F006A0375F005A4F8C5F0600278FFC3E89578
:10083F00645002A864886322C3E5409440E5419464
:10084F0001E5635003140158046002F563220208A6
:10085F00602275E890227883E6FFE5E820ECF7A8A0
:0F086F00BDA9BE0570C3E57094084052757000B6
:10087E00E9FA79A0E76044EA7007E571601B0208A7
:10088E009BC3E895716010E5715006600C14020868
:10089E00A70460F90208A7E571F571C3946D401BBA
:1008AE007561C0C394044013756180C39404400BFA
:1008BE00756140C39404400375610075BB0822E561
:1008CE0061F460020561E570B4070375BB10227414
:1008DE003279A787F0A4C5F0A2F733F8C3E8956183
:1008EE004002A8618822882488258826886422757B
:1008FE0040007541F022C2AF75C820A8CCA9CDAA80
:10090E003A30CF010A75C824D2AFAB3BAC3C883B22
:10091E00893CC3E89BF8E99C206908F930670241DD
:10092E0010216DAD3D8A3DF9EA9DFA600478FF799C
:10093E00FFAE3EAF3F8B3E8C3FA83BA93CC3E89E2B
:10094E00F8E99FF9C3E54113FBE54013FAE82AF5F0
:10095E0040E93BF54150067540FF7541FF21B7AAAE
:10096E0040AB41AC40AD417E047F02C3EB940440EA
:10097E00021E1FC3EB940840021E1FC3ED13FDECB5
:10098E0013FCDEF7C3EA9CFAEB9DFBEF6009C3E9AB
:10099E0013F9E813F8DFF7EA28FAEB39FB8A408BF4
:1009AE004150067BFF8B408B41C3EB94025002D229
:1009BE00673069047F0321E27892E6FFC3E537943E
:1009CE008240110FC3E53794A040010FC3EF940688
:1009DE0040027F057E02E541C4540FF9E541C4543F
:1009EE00F0F8E540C4540F28F8C3E89EFAE99400E5
:1009FE00FB4009C3EA9402EB940050047A02E4FB34
:100A0E00415CAA40AB41EBC4FEEAC4540F4EFCC39A
:100A1E00EA9CFAEB9400FBC3E813C313F8EA28FA36
:100A2E00EB3400FB8A408B41C3EB94024002C26759
:100A3E007802EBC4FE7B00EAC4540F4EFAC3EA9868
:100A4E00FA4005C3940250027A027892E6FF3060B3
:100A5E0002415C855192855293D26043E680C3E495
:100A6E009AF8E49BF930670241E8E8FAE9FBD3E92A
:100A7E0013FDE813FC88518952C3EF94036038EFDD
:100A8E0020E00DE82CF8E93DF9ECFAEDFB020AB195
:100A9E00E828F8E939F9C3E82402F8E93400F97ACC
:100AAE00FE7BFFC3EF9403400E8A538B54884D890F
:100ABE004E8C4F8D50611C885389548A4D8B4E8CB1
:100ACE004F8D503069127553F07554FF754FF07598
:100ADE0050FF7551F07552FF611CE8FAD3E813FC14
:100AEE008851C3EF94036020EF20E007E82CF8EC68
:100AFE00FA6108E8282402F87AFEC3EF940340084E
:100B0E008A53884D8C4F611C88538A4D8C4FE568F3
:100B1E00C3335002646BF56830600261267534028F
:100B2E00D26043E680E52D54066034A840A941C347
:100B3E00E913F9E813F8C3E913F9E813F830690477
:100B4E00E92440F9C2AF53E67F759100C3E498F5EE
:100B5E0094E499F595759104D26043E680D2AF2264
:100B6E00D265754300752000306C03752040020B72
:100B7E008DD265754300752040306C03752000786A
:100B8E00017901206720E52D54066002C2657914B3
:100B9E00E541C313700104F8C39414400278143075
:100BAE006904781B791B206010E543600C306903E3
:100BBE00D53404D26D812F712E0543E59B5440B57B
:100BCE002002811930690908C3E89940011861B4FF
:100BDE0020650A08C3E8994002618D61B4C265C2FE
:100BEE00AF53E67F7591003067127594007595FED0
:100BFE00759104D26043E680D2AF618DAE40AF41B5
:100C0E00C3E49EF594E49FF59561FEC3E53394012C
:100C1E005002618D306502618DD802812D61B4C2A2
:100C2E006DC2AF53E67F75910085539485549575CB
:100C3E009104854D92854E93D26043E680D2AFE506
:100C4E002D54066008206A020533020C6B306D0DC0
:100C5E00206C0A2065071581158102150722780080
:0F0C6E003064053065027801E53775F007A4F9A9
:100C7D00E5F028F5F0E9A2F013A2F113A2F213F5B5
:100C8D0037C394785003753778C3E53795384008E6
:100C9D00D266D295D293D29730600281A5854F92BC
:100CAD00855093D26043E68022207D16C2AF7542F7
:100CBD0002C296D294306202C293D2AF759F1102D6
:100CCD000EA5C2AF754202C296D292306202C29593
:100CDD00D2AF759F11020EA5307243207D20C2AF99
:100CED00754203900138757B40D293C292306204F5
:100CFD00C297A103D296D2AF759F13020EA5C2AFB4
:100D0D00754203900138757B40D295C294306204D0
:100D1D00C297A123D296D2AF759F10020EA5207D4A
:100D2D0017C2AF754203900113D293306202C2977E
:100D3D00D2AF759F13020EA5C2AF7542039001137A
:100D4D00D295306202C297D2AF759F10020EA520C8
:100D5D007D16C2AF754204C294D292306202C29720
:100D6D00D2AF759F10020EA5C2AF754204C292D2CA
:100D7D0094306202C297D2AF759F13020EA53072E6
:100D8D0043207D20C2AF754205900127757B10D29F
:100D9D0097C296306204C295A1A9D294D2AF759F25
:100DAD0011020EA5C2AF754205900149757B04D2A3
:100DBD0097C296306204C293A1C9D292D2AF759FE9
:100DCD0011020EA5207D17C2AF754205900109D203
:100DDD0097306202C295D2AF759F11020EA5C2AFB8
:100DED0075420590011DD2973062EBC293D2AF755B
:100DFD009F11020EA5207D16C2AF754206C292D27A
:100E0D0096306202C295D2AF759F13020EA5C2AF86
:100E1D00754206C294D296306202C293D2AF759FCC
:100E2D0010020EA5307243207D20C2AF7542019095
:100E3D000149757B04D295C294306204C293C14FAF
:100E4D00D292D2AF759F10020EA5C2AF754201901E
:100E5D000127757B10D293C292306204C295C16F87
:100E6D00D294D2AF759F13020EA5207D17C2AF7518
:100E7D00420190011DD295306202C293D2AF759F8F
:100E8D0010020EA5C2AF754201900109D2933062D6
:100E9D0002C295D2AF759F13C26622900107757B72
:100EAD0000D295D293D297C294C292C296C26222B8
:100EBD00788076FF0876FF0876FF0876FF087603C0
:100ECD0008760408760A0876030876010876017814
:100EDD008C76010876FF0876FF0876FF0876FF0806
:100EED0076FF0876030876FF0876FF0876FF08760A
:100EFD00250876D00876FA0876FA0876040876FF83
:100F0D0008760108760008767A0876FF08760108DB
:100F1D007601087600087603087600227887E6FFCA
:100F2D00C272BF0302D2727888E6C394036008C20E
:100F3D007DE630E102D27DC27E7889E630E102D2D3
:100F4D007EC3EF94026008758E01D273020F617536
:100F5D008E00C273227880E6149000809378A5F6F7
:100F6D007881E6149000809378A6F67886E6149042
:100F7D00008D9378A7F67886E6F539C39402500371
:100F8D00753902789CE67538FFB402037538A0B444
:100F9D00030375388278A3E61490009A93F566D111
:100FAD00A822227896E6FA7897E6FB7888E6B403CD
:100FBD0005C3EB940EFB307F047A007BFFC3EB9AE5
:100FCD00FCC3948250027C827572000572EC8572AE
:100FDD00F0A4C3E5F0947D40F222D27FF1B012056A
:100FED00A37A007B007C10120599E55C2AFA740047
:100FFD003BFBDCF37C04C3EB13FBEA13FADCF7FEDB
:10100D00C27F120FB022E5EF20E603752000052008
:10101D00903FFFE520146006901DFF1460009304BF
:10102D00600375EF1253D9BF7581C043FF80120560
:10103D009475EF0243B203E5B3240220E70DF521C9
:10104D00E5E320E0068521B343E301120EA8758088
:10105D00FF75A40075F1B275D4DF7590A975A5FC67
:0F106D0075F2FE75D50175A60175E241120EA848
:10107C00E4F8F6D8FD756801120EBD121558789873
:10108C008673753001C2AF1205AD1205BD1205A3F2
:10109C001205C41205A31205CB1205A31216711268
:1010AC0005AD1205AD1205A8C2AF78FA79FA3085F4
:1010BC0007D9FBD8F7021C00120F29120F62120F6E
:1010CC00AF120FB078988673120EA87588107589B8
:1010DC000275C82475910475D84075A82275B8029C
:1010EC0075E690759B80759D0075D10E75BC587515
:1010FC00BB0875BA1175E880120594D2AF12085D61
:10110C0075360053DACF207E0343DA20307E03435A
:10111C00DA1043DA01C2D8C2711205ADD2617B0379
:10112C007A0CE55B70077A0CDB030210B41205A392
:10113C002070030210B4C270E55CC3940240E1E578
:10114C002F541F855E5DF55EB55DD5DAD5C2615352
:10115C00DACF207E0343DA20307E0343DA10C2D884
:10116C00C27178A2E67008D274E52F54E0F52FC254
:10117C00757529001205A8307409C3E529940A4035
:10118C0002D27512059978023074027800C3E55CBE
:10119C009840F0C2AF1205BD1205BD1205BDD2AF0D
:1011AC001205AD754C007888E6B403024197120520
:1011BC0099788CE6C394015003021297E530C394DE
:1011CC00015003021297207435C3E55C94FF500361
:1011DC00021297C2AF1205D2D2AF1205A8C3E55CBA
:1011EC00940150EFC2AF1205BD12059E1205BDD27F
:1011FC00AF1205A8C3E55C94FF40E90216F67F0523
:10120C00D27F120FB01205A8C2AFC27F120FB0AEC0
:10121C005CC3E55C947FD2AF407B120594C2AF12E5
:10122C0005D2D2AFDFDA120FE7C3EE94057897F64A
:10123C001205AD12159A1216797F0AD27F120FB0D1
:10124C001205A8C2AFC27F120FB0AE5CC3E55C94AE
:10125C007FD2AF50E4120594C2AF1205BD12059EA9
:10126C001205BDD2AFDFD4120FE7EE24037896F649
:10127C001205AD12159A1216A81205A8120FB0C3BA
:10128C00E55C94FF500221D20216F6C3E55C954C46
:10129C004003855C4C1205A878017988E7B40302F9
:1012AC007805C3E55C98400221B2C2AF1205D21298
:1012BC0005D21205D2D2AF1205AD753000E4F5316E
:1012CC00F5320531E531F4703F0532789AE678193C
:1012DC00146012783214600D787D14600878FA145A
:1012EC006003753200C3E53298401D120EA812053A
:1012FC0094153275310078998673C2AF1205D2D22B
:10130C00AF789886731205A812059EE52A700530F1
:10131C00740201B478012074027806C3E55C98402D
:10132C00A17888E6C3940360031205A8E52A70032C
:10133C000210B4C2AF120EA8E4F522F523F524F581
:10134C0025F526F567D2AF7885E6C333F565E4F568
:10135C0044F545F546F547F548F570F52CF52DF5B2
:10136C003775700875BB10120594120861E5E820FA
:10137C00ECFBA8BDA9BEE97001F88871120865756F
:10138C00700875BB10120F29C2AF7561FF1208DD12
:10139C00852261852262852263D2AF752201752474
:1013AC0001752501752601856069756A017888E6E5
:1013BC00B40307C27D307602D27DD268D269753310
:1013CC0000120E02120E311208FD1209041208FD51
:1013DC001209041208FD120B7F1206AD120C6C12CE
:1013EC000CB6120904120B6E306E031206AE206797
:1013FC0003120800306703120847120C6C120CE53C
:10140C00120904120B7F306E031206EA120C6C12D6
:10141C000D5C120904120B6E306E03120748120C8D
:10142C006C120D8B120904120B7F306E031207A580
:10143C00120C6C120E02120904120861120B6E12BD
:10144C000C6C120E3112086512090430692F856478
:10145C0061856462856069756A0179187A0CC3E5E7
:0D146C003399400CC269D26A8A357561FF60
:10147900021489C3E55C940140030213E202150FCB
:10148900306A1D206C1AE535147006C26AD26B6188
:10149900E2F535C3E55C940140030213E202150F3E
:1014A900753600788279A4E760027803C3E55F980E
:1014B9005054307404E52A604D7888E6B403172047
:1014C9007D0520760781DF30760281DF206C07D227
:1014D9006C856461812178F0306C058564617820C0
:1014E900C3E54198500261E2306C1BC26CC27D3089
:1014F9007602D27DD26A75351285646161E205365C
:10150900E55C6002A112753600C2AF120EA8788799
:10151900E6FE7602120F297887EEF6E4F522F52326
:10152900F524F525F526F565752C00752D00D2AF46
:101539001205A8120EA878A4E66006C295C297C241
:1015490093307409C3E5369404400201B441C9904B
:101559001A0D78201215DCE520B45A0CA31215DCFB
:10156900E520B4A50302157A120EBD12159A0215CB
:1015790099901A0378807B0A1215DCA308DBF9908D
:101589001A0F788C7B191215DCA308DBF9901A283D
:1015990022C2AF12161B1215F5901A00740E1215FD
:1015A900E1A374061215E1A374151215E1901A034B
:1015B90078807B0A1215E0A308DBF9901A0F788C62
:1015C9007B191215E0A308DBF912162E12160C90DE
:1015D9001A2822E493F622E6438F01538FFD75EF13
:1015E9000275B7A575B7F1F0538FFE22438F0243F9
:1015F9008F0175EF0275B7A575B7F1901A0DF05304
:101609008FFC22901A0D745AB1E1901A0E74A5B18B
:10161900E1227A3079D07820901A40B1DCE520F7C0
:1016290009A3DAF7227A3079D0901A40E7B1E109B3
:10163900A3DAF922AB74A875BB01027984BB020253
:101649007985BB03027986BB04027992BB050279CD
:1016590087BB060279A3BB0702799CBB080279887C
:10166900BB09027989E8F7227C051205ADDCFB226A
:10167900C2AF1205BD1205C41205CB1205D212055F
:101689009E1205BD1205C41205CB1205D212059E84
:101699001205BD1205C41205CB1205D2D2AF22C262
:1016A900AF1205D21205CB1205C41205BD12059E53
:1016B9001205D21205CB1205C41205BD12059E12E0
:1016C90005D21205CB1205C41205BDD2AF22AE74E4
:1016D900AF75C2AF1205BD1205BD1205BD12059E3B
:1016E900DEF21205D212059EDFF8D2AF22D179D1EE
:1016F90071D171757401757501757600D1D77C0545
:10170900AD5C1205ADC3ED955C70F5C3E55C940164
:10171900400AC3E55C94FF4032021732D13DB19AC9
:10172900D179C2AF75EF12D171DCD50576C3E576F3
:101739009403500280C6D1710575E5741490009F19
:1017490093F808C3E57598500280AED171D171053F
:1017590074C3E574940A5002809C120EBDB19AC2FA
:06176900AF75EF12D17113
:0319FD00021013C2
:101A00000E0615FFFFFFFF03040A0301015AA5019B
:101A1000FFFFFFFFFF03FFFFFF25D0FAFA04FF01DE
:091A2000007AFF0101000300FF40
:101A4000235475726E6967794E6665743235412329
:101A500023424C48454C4923463333302320202031
:101A60002020202020202020202020202020202076
:101C0000C2AFC2D353D9BF7581C043B20343FF8073
:101C1000752438752503B1C975EF0275E24043F1AB
:101C20002053A4DF75D4FFD2857DFA780379E67C52
:101C300010752200752300901DD67B0675249875BB
:101C400025013085028142208508D8FBD9F9DCF7CF
:101C500081B4308508D8FBD9F9DCF781B4B189E4C7
:101C600093A3C39A6004DDC381B4DBDBB17B600264
:101C7000812B7B08E493FAA3B15CDBF87A30B15C8A
:101C8000752200752300B17BEAFCEBFDC3ED94FEE9
:101C9000400EB17B8A278B28ED30E0048A828B834B
:101CA000B17B7AC270D8C3ED94FE601350CEBD00F4
:101CB00025EC60097520007521FF0200008100A855
:101CC00027A9280809D804D90281D3B17FEA89AAB3
:101CD000F281C50D81A0C3ED94035049EDA2E092BD
:101CE000007AC5C3E5829400E583941C50902000DF
:101CF00010438F02438F0175B7A575B7F1F030001F
:101D00001FA827A9280809438F01538FFDD804D99C
:101D100002A12089AAE275B7A575B7F1F0A3A10DBC
:101D2000538FFC817C7AC1BD030CE493A3FAB140CC
:101D3000DCF8B138817C817EAA22AB23B15CEBFA5E
:101D4000EA6222752608C3E52313F523E52213F57D
:101D50002250066323A0632201D526EAB1C9B1C986
:101D600075260AEAF4200102D285300102C285B14B
:101D7000C9C3134002C201D526EB22B17FEAFB2082
:101D80008502A17F308502A184752608AE24AF2587
:101D9000C3EF13FFEE13FEB1CDB1C9C3EA13308513
:101DA000024480FA30E703632201C3E52313F523DD
:101DB000E52213F52250066323A0632201D526D91C
:101DC000E52265236523F52222AE24AF250E0FDE22
:101DD000FEDFFCD20122424C48656C693437316326
:041DE000F3300601D5
:00000001FF
